:03000000020100FA
:03000B0002015996
:1001000075A7167880E4F6D8FD75F67E5385814391
:10011000847C75AD287589117D0A7E0FC281C294D9
:10012000D2C7D28CD2A9438502439210208702D233
:1001300007D2AFC29375A61E75A6E131787400711F
:1001400043F52174017143F52274027143F5237460
:10015000037143F524318480DCC0D0DE047E0FD2ED
:1001600078DB127B0530050D300006C200C293809B
:1001700004D200D293D0D032E5AD20E104DD04D228
:10018000057D0A22E521207806B5250302019AF5AE
:1001900025752900208001F431DFE522207806B59D
:1001A00026030201B0F526752901209701F431DFFD
:1001B000E523207806B527030201C6F52775290235
:1001C000209601F431DFE524207806B528030201EA
:1001D000DCF528752903209501F431DFC27822F57A
:1001E0002A711C51D5C2AFD2817C485181790171ED
:1001F0007E304905517D0201FB51A9304805517DF2
:1002000002020551A9305005517D02020F51A9305B
:100210005105517D02021951A9305205517D02024A
:100220002351A9305305517D02022D51A9305405A7
:10023000517D02023751A9305505517D02024151CD
:10024000A9305605517D02024B51A9305705517D09
:1002500002025551A9305905517D02025F51A93062
:100260005805517D02026951A9300205517D0202F3
:100270007351A951A9D2AF300702717C22D2817C7F
:1002800012300702D29400000000000000000000BD
:10029000000000C294000000000000000000000008
:1002A000DCDFC2817901717E22D2817C12300702AB
:1002B000D29400000000000000000000000000C216
:1002C000940000000000000000000000DCDFC2819C
:1002D000747D718522740030490224013048022463
:1002E0000130570224013056022401305502240106
:1002F00030540224013053022401305202240130D0
:100300005102240130500224013059022401305896
:1003100002240120E003C20222D2022220900E20F9
:10032000030DD203E52B6401F52B02032FC203203A
:10033000910E20040DD204E52B6402F52B0203423A
:10034000C204227904752C00752D0042C0F52ED20E
:10035000C330C4FDE5C5C2C453C0FC252CF52CE553
:100360002D3400F52DE52ED9E2C3E52D13F52DE54D
:100370002C13F52CC3E52D13E52C1322790A74FAFE
:0B0380007185D9FA220000D5E0FB22B5
:00000001FF
